:020000040000FA
:0A0000000000000035EF00F041D0D1
:080018008ED0076A066EFF0E90
:100020000626072200D0D8A01200030E056EE60EA9
:1000300002D8F5D7056AFE0F046EE86A055AD8A003
:1000400012000000040600D0F8D706500A02F3CFD1
:1000500008F0F4CF09F007500A02F35009260650C1
:100060000B02F3500926085012004F0EAF6E240EFB
:10007000AC6E900EAB6E0001C69AC00E926E936A83
:10008000946E0F0EC16E070EB46E6CD0F2A403D046
:10009000F294827011009EAA19D0060EAB1412E1E0
:1000A000E2CF14F0E1CF13F0152A11EE00F0155055
:1000B000E126000EE222AECFE7FF14C0E2FF13C03C
:1000C000E1FF1100AE50AE50AB98AB881100155057
:1000D000165C14E0162AEACF05F0E9CF04F001EE31
:1000E00000F01650E926000EEA22EF50046E05C01B
:1000F000EAFF04C0E9FFD880120004D0E868046E6B
:10010000D8A012001200156A166A9D8A9F8AF28E84
:10011000F28C12009D9A01EE00F0010EF46EF36A6B
:10012000F306000EF45AEE6AF450F310F9E1156A82
:10013000166A9D8A1200F29EE0CF8DF4D8CF8EF41D
:10014000E8CF8FF4F28E0001A192F29E8DC4E0FF01
:100150008EC4D8FF8FC4E8FFF28E10009EA8FED791
:10016000AD6E1200929489949292898292908990B5
:100170009296898692988998929A898A939E8A9E65
:10018000939C8A8C939A8A9A93988A8893968A9653
:1001900093948A8493928A9293908A80949A8B9A69
:1001A00094988B8894928B9294948B94320E35DF32
:1001B0009292899292968996929A899A939C8A9C15
:1001C00093988A9893948A9493908A9094988B9811
:1001D0004B6A4A6A4D6A4C6A4F6A4E6A516A506A63
:1001E000536A526A556A546A576A566A596A586A13
:1001F000616A626A636A646A656A666A676A686A8B
:10020000236A896B8A6BFEEC0DF01DEC0EF0226AFE
:10021000216A206A936A8A6A76DF7CDFCD6AF2946B
:10022000F28A870ED56EB16AA192B368E20EB26E01
:1002300000EE69F0200EEE68E82EFDD75E685D8E58
:10024000276A266A256A246A282AE86A28B2010FE2
:1002500029B0010806E12970242A000E2522262251
:10026000272235DF176EBC0E175C06E3FE0E175C07
:10027000D8A0196A82EF07F017AE20D0196A8B0E4A
:10028000175C04E117C019F01A6814D09B0E175CB4
:1002900004E117C019F01C680DD0AB0E175C04E127
:1002A00017C019F01E6806D0BB0E175C03E117C01B
:1002B00019F05F6882EF07F080EF07F0195204E150
:1002C00082EF07F080EF07F08B0E195CD8A459D1AC
:1002D0001A2805E117C01AF082EF07F050D117C0B5
:1002E0001BF0240E1A5C26E122901B5222E0899416
:1002F00002EE8DF0D8901B34E926000EEA22EECFF4
:100300003AF0EFCF3BF03A502424006E3B502520CA
:10031000016E000E2620026E000E2720036E03C021
:100320006CF002C06BF001C06AF000C069F0208080
:10033000898222D1250E1A5C26E122921B5222E0EC
:10034000899002EE8DF0D8901B34E926000EEA2247
:10035000EECF3CF0EFCF3DF03C502424006E3D50FA
:100360002520016E000E2620026E000E2720036E4F
:1003700003C070F002C06FF001C06EF000C06DF0FD
:1003800020828986F9D0260E1A5C26E122941B521F
:1003900022E0899802EE8DF0D8901B34E926000EF9
:1003A000EA22EECF3EF0EFCF3FF03E502424006E25
:1003B0003F502520016E000E2620026E000E2720E1
:1003C000036E03C074F002C073F001C072F000C08D
:1003D00071F02084898AD0D0270E1A5C26E12296FB
:1003E0001B5222E08A9E02EE8DF0D8901B34E92643
:1003F000000EEA22EECF40F0EFCF41F0405024242F
:10040000006E41502520016E000E2620026E000E67
:100410002720036E03C078F002C077F001C076F0A9
:1004200000C075F020868A8CA7D0280E1A5C26E1C1
:1004300022981B5222E08A9A02EE8DF0D8901B344B
:10044000E926000EEA22EECF42F0EFCF43F0425011
:100450002424006E43502520016E000E2620026EDB
:10046000000E2720036E03C07CF002C07BF001C0A9
:100470007AF000C079F020888A887ED0290E1A5C34
:1004800026E1229A1B5222E08A9602EE8DF0D89045
:100490001B34E926000EEA22EECF44F0EFCF45F000
:1004A00044502424006E45502520016E000E262065
:1004B000026E000E2720036E03C080F002C07FF0A2
:1004C00001C07EF000C07DF0208A8A8455D02A0EBB
:1004D0001A5C26E1229C1B5222E08A9202EE8DF0E9
:1004E000D8901B34E926000EEA22EECF46F0EFCF7B
:1004F00047F046502424006E47502520016E000E20
:100500002620026E000E2720036E03C084F002C076
:1005100083F001C082F000C081F0208C8A802CD052
:100520002B0E1A5C26E1229E1B5222E08B9A02EED1
:100530008DF0D8901B34E926000EEA22EECF48F069
:10054000EFCF49F048502424006E49502520016E19
:10055000000E2620026E000E2720036E03C088F0D6
:1005600002C087F001C086F000C085F0208E8B8825
:1005700003D01A6882EF07F01A6880EF07F080EF67
:1005800007F09B0E195CD8A4AFEF06F01C2804E11D
:1005900017C01CF0AEEF06F017C01DF01D52D8A416
:1005A0005ED0240E1C5C08E1229020B004D06C6860
:1005B0006B686A68696850D0250E1C5C08E122925D
:1005C00020B204D070686F686E686D6845D0260EE2
:1005D0001C5C08E1229420B404D0746873687268CB
:1005E00071683AD0270E1C5C08E1229620B604D030
:1005F00078687768766875682FD0280E1C5C08E1EB
:10060000229820B804D07C687B687A68796824D006
:10061000290E1C5C08E1229A20BA04D080697F6808
:100620007E687D6819D02A0E1C5C08E1229C20BCE3
:1006300004D084698369826981690ED02B0E1C5CA9
:1006400008E1229E20BE04D0886987698669856991
:1006500003D01C6882EF07F01C6880EF07F0240EBF
:100660001C5CD8A46CD0898402EE8DF0D8901D3427
:10067000E926000EEA22EECF2AF0EFCF2BF03B6AFC
:100680003A6A20802A502424006E2B502520016EC7
:10069000000E2620026E000E2720036E03C06CF0B1
:1006A00002C06BF001C06AF000C069F06152D8B4BA
:1006B00043D0228002EE8DF0D8908A35E926000ED4
:1006C000EA22EECF8BF0EFCF8CF02A508B5D2B50CF
:1006D0008C5904E22BC08CF02AC08BF02A508B2757
:1006E0002B508C23D8908B378C3703EE8DF0D8901D
:1006F0006134E926000EEA22EECF00F0EFCF01F0E0
:1007000000508B5D01508C5905E38CC04BF08BC0C1
:100710004AF011D003EE8DF0D8906134E926000E36
:10072000EA22EECF00F0EFCF01F08B51005C4A6E71
:100730008C5101584B6E01D02290ACEF06F0250E83
:100740001C5CD8A46CD0898002EE8DF0D8901D344A
:10075000E926000EEA22EECF2CF0EFCF2DF03D6A15
:100760003C6A20822C502424006E2D502520016EDE
:10077000000E2620026E000E2720036E03C070F0CC
:1007800002C06FF001C06EF000C06DF06252D8B4CC
:1007900043D0228202EE8DF0D8908A35E926000EF1
:1007A000EA22EECF8BF0EFCF8CF02C508B5D2D50EA
:1007B0008C5904E22DC08CF02CC08BF02C508B2770
:1007C0002D508C23D8908B378C3703EE8DF0D8903A
:1007D0006234E926000EEA22EECF00F0EFCF01F0FE
:1007E00000508B5D01508C5905E38CC04DF08BC0DF
:1007F0004CF011D003EE8DF0D8906234E926000E53
:10080000EA22EECF00F0EFCF01F08B51005C4C6E8E
:100810008C5101584D6E01D02292ACEF06F0260E9D
:100820001C5CD8A46CD0898802EE8DF0D8901D3461
:10083000E926000EEA22EECF2EF0EFCF2FF03F6A2E
:100840003E6A20842E502424006E2F502520016EF5
:10085000000E2620026E000E2720036E03C074F0E7
:1008600002C073F001C072F000C071F06352D8B4DE
:1008700043D0228402EE8DF0D8908A35E926000E0E
:10088000EA22EECF8BF0EFCF8CF02E508B5D2F5005
:100890008C5904E22FC08CF02EC08BF02E508B2789
:1008A0002F508C23D8908B378C3703EE8DF0D89057
:1008B0006334E926000EEA22EECF00F0EFCF01F01C
:1008C00000508B5D01508C5905E38CC04FF08BC0FC
:1008D0004EF011D003EE8DF0D8906334E926000E6F
:1008E000EA22EECF00F0EFCF01F08B51005C4E6EAC
:1008F0008C5101584F6E01D02294ACEF06F0270EB8
:100900001C5CD8A46BD08A8E02EE8DF0D8901D347A
:10091000E926000EEA22EECF30F0EFCF31F0416A47
:10092000406A208630502424006E31502520016E0C
:10093000000E2620026E000E2720036E03C078F002
:1009400002C077F001C076F000C075F06452D8B4F0
:1009500043D0228602EE8DF0D8908A35E926000E2B
:10096000EA22EECF8BF0EFCF8CF030508B5D315020
:100970008C5904E231C08CF030C08BF030508B27A2
:1009800031508C23D8908B378C3703EE8DF0D89074
:100990006434E926000EEA22EECF00F0EFCF01F03A
:1009A00000508B5D01508C5905E38CC051F08BC019
:1009B00050F011D003EE8DF0D8906434E926000E8B
:1009C000EA22EECF00F0EFCF01F08B51005C506EC9
:1009D0008C510158516E01D02296BED1280E1C5C5C
:1009E000D8A46BD002EE8DF0D8901D34E926000E0D
:1009F000EA22EECF32F0EFCF33F0436A426A8A8ABE
:100A0000208832502424006E33502520016E000EC1
:100A10002620026E000E2720036E03C07CF002C069
:100A20007BF001C07AF000C079F06552D8B443D0B1
:100A3000228802EE8DF0D8908A35E926000EEA224F
:100A4000EECF8BF0EFCF8CF032508B5D33508C5962
:100A500004E233C08CF032C08BF032508B2733501D
:100A60008C23D8908B378C3703EE8DF0D89065347B
:100A7000E926000EEA22EECF00F0EFCF01F00050A1
:100A80008B5D01508C5905E38CC053F08BC052F044
:100A900011D003EE8DF0D8906534E926000EEA22DD
:100AA000EECF00F0EFCF01F08B51005C526E8C5115
:100AB0000158536E01D022984FD1290E1C5CD8A446
:100AC0006BD002EE8DF0D8901D34E926000EEA229C
:100AD000EECF34F0EFCF35F0456A446A8A86208A3B
:100AE00034502424006E35502520016E000E26203F
:100AF000026E000E2720036E03C080F002C07FF05C
:100B000001C07EF000C07DF06652D8B443D0228A86
:100B100002EE8DF0D8908A35E926000EEA22EECF5B
:100B20008BF0EFCF8CF034508B5D35508C5904E254
:100B300035C08CF034C08BF034508B2735508C236B
:100B4000D8908B378C3703EE8DF0D8906634E92639
:100B5000000EEA22EECF00F0EFCF01F000508B5DE7
:100B600001508C5905E38CC055F08BC054F011D066
:100B700003EE8DF0D8906634E926000EEA22EECF1F
:100B800000F0EFCF01F08B51005C546E8C51015896
:100B9000556E01D0229AE0D02A0E1C5CD8A46BD0EE
:100BA00002EE8DF0D8901D34E926000EEA22EECF39
:100BB00036F0EFCF37F0476A466A8A82208C36508B
:100BC0002424006E37502520016E000E2620026E70
:100BD000000E2720036E03C084F002C083F001C022
:100BE00082F000C081F06752D8B443D0228C02EE6C
:100BF0008DF0D8908A35E926000EEA22EECF8BF0F0
:100C0000EFCF8CF036508B5D37508C5904E237C0F3
:100C10008CF036C08BF036508B2737508C23D89011
:100C20008B378C3703EE8DF0D8906734E926000EB1
:100C3000EA22EECF00F0EFCF01F000508B5D0150C3
:100C40008C5905E38CC057F08BC056F011D003EEE1
:100C50008DF0D8906734E926000EEA22EECF00F03E
:100C6000EFCF01F08B51005C566E8C510158576EDE
:100C700001D0229C71D02B0E1C5CD8A46BD002EE4C
:100C80008DF0D8901D34E926000EEA22EECF38F020
:100C9000EFCF39F0496A486A8B8A208E3850242475
:100CA000006E39502520016E000E2620026E000EC7
:100CB0002720036E03C088F002C087F001C086F0D1
:100CC00000C085F06852D8B443D0228E02EE8DF079
:100CD000D8908A35E926000EEA22EECF8BF0EFCFCE
:100CE0008CF038508B5D39508C5904E239C08CF04F
:100CF00038C08BF038508B2739508C23D8908B37E5
:100D00008C3703EE8DF0D8906834E926000EEA2285
:100D1000EECF00F0EFCF01F000508B5D01508C5909
:100D200005E38CC059F08BC058F011D003EE8DF064
:100D3000D8906834E926000EEA22EECF00F0EFCF1B
:100D400001F08B51005C586E8C510158596E01D0E6
:100D5000229E02D01C68D6D01C68D2D0D1D0AB0E57
:100D6000195CD8A4C0D01E2804E117C01EF0CAD058
:100D7000B9D0240E1E5C14E117C061F061520CE082
:100D800003EE8DF0D8906134E926000EEA22EECF12
:100D90004AF0EFCF4BF003D04B6A4A6A2290A0D0C2
:100DA000250E1E5C14E117C062F062520CE003EEE7
:100DB0008DF0D8906234E926000EEA22EECF4CF096
:100DC000EFCF4DF003D04D6A4C6A229289D0260EA7
:100DD0001E5C14E117C063F063520CE003EE8DF06B
:100DE000D8906334E926000EEA22EECF4EF0EFCF22
:100DF0004FF003D04F6A4E6A229472D0270E1E5CC9
:100E000014E117C064F064520CE003EE8DF0D8904A
:100E10006434E926000EEA22EECF50F0EFCF51F015
:100E200003D0516A506A22965BD0280E1E5C14E1F2
:100E300017C065F065520CE003EE8DF0D890653474
:100E4000E926000EEA22EECF52F0EFCF53F003D0A6
:100E5000536A526A229844D0290E1E5C14E117C0CE
:100E600066F066520CE003EE8DF0D8906634E92609
:100E7000000EEA22EECF54F0EFCF55F003D0556AC2
:100E8000546A229A2DD02A0E1E5C14E117C067F016
:100E900067520CE003EE8DF0D8906734E926000E1F
:100EA000EA22EECF56F0EFCF57F003D0576A566ADA
:100EB000229C16D02B0E1E5C13E117C068F06852FE
:100EC0000CE003EE8DF0D8906834E926000EEA229B
:100ED000EECF58F0EFCF59F003D0596A586A229EEE
:100EE0001E6810D00DD0BB0E195C0AE15F2804E12A
:100EF00017C05FF007D004D017C060F0F9EC0CF019
:100F0000BFEC0CF0080E5E5CD8B0B6EF0CF05A5097
:100F1000245C5B5025585C5026585D502758D8A05B
:100F200096EF0CF05D8E5E52D8A49DD022B038D0E2
:100F30003B503A102CE18994208002EE8DF0D8903D
:100F40008A35E926000EEA22EECF3AF0EFCF3BF0E9
:100F50002A503A5C2B503B5804E22BC03BF02AC08D
:100F60003AF03A502424006E3B502520016E000ECA
:100F70002620026E000E2720036E03C06CF002C014
:100F80006BF001C06AF000C069F0898208D08992D4
:100F900020906C686B686A6869683B6A3A6A61D0DD
:100FA00020A047D03B503A102BE1899402EE8DF0FF
:100FB000D8908A35E926000EEA22EECF3AF0EFCF3C
:100FC0003BF02A503A5C2B503B5804E22BC03BF0DC
:100FD0002AC03AF03A502424006E3B502520016E7E
:100FE000000E2620026E000E2720036E03C06CF058
:100FF00002C06BF001C06AF000C069F0898218D0AD
:1010000089924A502424006E4B502520016E000E18
:101010002620026E000E2720036E03C06CF002C073
:101020006BF001C06AF000C069F020903B6A3A6A38
:1010300018D089842A502424006E2B502520016E5C
:10104000000E2620026E000E2720036E03C06CF0F7
:1010500002C06BF001C06AF000C069F020803B6AFA
:101060003A6A95EF0CF0010E5E5CD8A49DD022B2D6
:1010700038D03D503C102CE18990208202EE8DF05A
:10108000D8908A35E926000EEA22EECF3CF0EFCF69
:101090003DF02C503C5C2D503D5804E22DC03DF0FD
:1010A0002CC03CF03C502424006E3D502520016EA5
:1010B000000E2620026E000E2720036E03C070F083
:1010C00002C06FF001C06EF000C06DF0898608D0DC
:1010D0008996209270686F686E686D683D6A3C6A98
:1010E00061D020A247D03D503C102BE1899002EE08
:1010F0008DF0D8908A35E926000EEA22EECF3CF03A
:10110000EFCF3DF02C503C5C2D503D5804E22DC0FB
:101110003DF02CC03CF03C502424006E3D50252076
:10112000016E000E2620026E000E2720036E03C003
:1011300070F002C06FF001C06EF000C06DF08986E3
:1011400018D089964C502424006E4D502520016EF5
:10115000000E2620026E000E2720036E03C070F0E2
:1011600002C06FF001C06EF000C06DF020923D6AC9
:101170003C6A18D089802C502424006E2D502520E4
:10118000016E000E2620026E000E2720036E03C0A3
:1011900070F002C06FF001C06EF000C06DF02082F0
:1011A0003D6A3C6A95EF0CF0020E5E5CD8A49DD0BF
:1011B00022B438D03F503E102CE18998208402EEB2
:1011C0008DF0D8908A35E926000EEA22EECF3EF067
:1011D000EFCF3FF02E503E5C2F503F5804E22FC01F
:1011E0003FF02EC03EF03E502424006E3F5025209C
:1011F000016E000E2620026E000E2720036E03C033
:1012000074F002C073F001C072F000C071F0898AFE
:1012100008D0899A209474687368726871683F6A0C
:101220003E6A61D020A447D03F503E102BE1899800
:1012300002EE8DF0D8908A35E926000EEA22EECF34
:101240003EF0EFCF3FF02E503E5C2F503F5804E26F
:101250002FC03FF02EC03EF03E502424006E3F5081
:101260002520016E000E2620026E000E2720036E40
:1012700003C074F002C073F001C072F000C071F0DE
:10128000898A18D0899A4E502424006E4F50252008
:10129000016E000E2620026E000E2720036E03C092
:1012A00074F002C073F001C072F000C071F02094BD
:1012B0003F6A3E6A18D089882E502424006E2F5031
:1012C0002520016E000E2620026E000E2720036EE0
:1012D00003C074F002C073F001C072F000C071F07E
:1012E00020843F6A3E6A95EF0CF0030E5E5CD8A442
:1012F0009DD022B638D0415040102CE18A9E2086E5
:1013000002EE8DF0D8908A35E926000EEA22EECF63
:1013100040F0EFCF41F03050405C3150415804E292
:1013200031C041F030C040F040502424006E4150A4
:101330002520016E000E2620026E000E2720036E6F
:1013400003C078F002C077F001C076F000C075F0FD
:101350008A8C08D08A9C2096786877687668756849
:10136000416A406A61D020A647D0415040102BE12D
:101370008A9E02EE8DF0D8908A35E926000EEA2288
:10138000EECF40F0EFCF41F03050405C315041584B
:1013900004E231C041F030C040F040502424006EDF
:1013A00041502520016E000E2620026E000E2720DF
:1013B000036E03C078F002C077F001C076F000C081
:1013C00075F08A8C18D08A9C50502424006E51509D
:1013D0002520016E000E2620026E000E2720036ECF
:1013E00003C078F002C077F001C076F000C075F05D
:1013F0002096416A406A18D08A8E30502424006EAC
:1014000031502520016E000E2620026E000E27208E
:10141000036E03C078F002C077F001C076F000C020
:1014200075F02086416A406A95EF0CF0040E5E5C10
:10143000D8A49CD022B838D0435042102CE18A9ACC
:10144000208802EE8DF0D8908A35E926000EEA2237
:10145000EECF42F0EFCF43F03250425C335043586E
:1014600004E233C043F032C042F042502424006E04
:1014700043502520016E000E2620026E000E27200C
:10148000036E03C07CF002C07BF001C07AF000C0A4
:1014900079F08A8808D08A9820987C687B687A6876
:1014A0007968436A426A61D020A847D0435042100D
:1014B0002BE18A9A02EE8DF0D8908A35E926000E4B
:1014C000EA22EECF42F0EFCF43F03250425C33508D
:1014D000435804E233C043F032C042F04250242467
:1014E000006E43502520016E000E2620026E000E75
:1014F0002720036E03C07CF002C07BF001C07AF0AD
:1015000000C079F08A8818D08A9852502424006E3E
:1015100053502520016E000E2620026E000E27205B
:10152000036E03C07CF002C07BF001C07AF000C003
:1015300079F02098436A426A18D08A8A325024246B
:10154000006E33502520016E000E2620026E000E24
:101550002720036E03C07CF002C07BF001C07AF04C
:1015600000C079F02088436A426ADFD1050E5E5CD4
:10157000D8A49CD022BA38D0455044102CE18A9689
:10158000208A02EE8DF0D8908A35E926000EEA22F4
:10159000EECF44F0EFCF45F03450445C3550455821
:1015A00004E235C045F034C044F044502424006EB9
:1015B00045502520016E000E2620026E000E2720C9
:1015C000036E03C080F002C07FF001C07EF000C057
:1015D0007DF08A8408D08A94209A80697F687E682A
:1015E0007D68456A446A61D020AA47D045504410BE
:1015F0002BE18A9602EE8DF0D8908A35E926000E0E
:10160000EA22EECF44F0EFCF45F03450445C355041
:10161000455804E235C045F034C044F04450242419
:10162000006E45502520016E000E2620026E000E31
:101630002720036E03C080F002C07FF001C07EF05F
:1016400000C07DF08A8418D08A9454502424006EFF
:1016500055502520016E000E2620026E000E272018
:10166000036E03C080F002C07FF001C07EF000C0B6
:101670007DF0209A456A446A18D08A863450242422
:10168000006E35502520016E000E2620026E000EE1
:101690002720036E03C080F002C07FF001C07EF0FF
:1016A00000C07DF0208A456A446A3FD1060E5E5C28
:1016B000D8A49CD022BC38D0475046102CE18A9246
:1016C000208C02EE8DF0D8908A35E926000EEA22B1
:1016D000EECF46F0EFCF47F03650465C37504758D4
:1016E00004E237C047F036C046F046502424006E6E
:1016F00047502520016E000E2620026E000E272086
:10170000036E03C084F002C083F001C082F000C009
:1017100081F08A8008D08A90209C846983698269DC
:101720008169476A466A61D020AC47D0475046106D
:101730002BE18A9202EE8DF0D8908A35E926000ED0
:10174000EA22EECF46F0EFCF47F03650465C3750F6
:10175000475804E237C047F036C046F046502424CC
:10176000006E47502520016E000E2620026E000EEE
:101770002720036E03C084F002C083F001C082F012
:1017800000C081F08A8018D08A9056502424006EC0
:1017900057502520016E000E2620026E000E2720D5
:1017A000036E03C084F002C083F001C082F000C069
:1017B00081F0209C476A466A18D08A8236502424D9
:1017C000006E37502520016E000E2620026E000E9E
:1017D0002720036E03C084F002C083F001C082F0B2
:1017E00000C081F0208C476A466A9FD0070E5E5C7D
:1017F000D8A49BD022BE38D0495048102CE18B9AF7
:10180000208E02EE8DF0D8908A35E926000EEA226D
:10181000EECF48F0EFCF49F03850485C3950495886
:1018200004E239C049F038C048F048502424006E22
:1018300049502520016E000E2620026E000E272042
:10184000036E03C088F002C087F001C086F000C0BC
:1018500085F08B8808D08B98209E88698769866977
:101860008569496A486A61D020AE47D0495048101E
:101870002BE18B9A02EE8DF0D8908A35E926000E86
:10188000EA22EECF48F0EFCF49F03850485C3950AB
:10189000495804E239C049F038C048F0485024247F
:1018A000006E49502520016E000E2620026E000EAB
:1018B0002720036E03C088F002C087F001C086F0C5
:1018C00000C085F08B8818D08B9858502424006E67
:1018D00059502520016E000E2620026E000E272092
:1018E000036E03C088F002C087F001C086F000C01C
:1018F00085F0209E496A486A18D08B8A3850242483
:10190000006E39502520016E000E2620026E000E5A
:101910002720036E03C088F002C087F001C086F064
:1019200000C085F0208E496A486A29D827AE1DD0AC
:10193000276A266A256A246A216A206A226A00EEDA
:1019400069F0200EEE68E82EFDD78994899289907F
:1019500089968998899A8A9E8A9C8A9A8A988A9670
:101960008A948A928A908B9A8B9806D027AE04D05C
:10197000276A266A256A246A827624EF01F05E6867
:101980005D8E186A080E185C33E2D8901834E96E40
:10199000EA6AEA36E936EA36690EE926000EEA22F4
:1019A000EFCF00F0ECCF01F0ECCF02F0ECCF03F082
:1019B0005A50005C5B5001585C5002585D5003580F
:1019C00015E2D8901834E96EEA6AEA36E936EA3662
:1019D000690EE926000EEA22EFCF5AF0ECCF5BF059
:1019E000ECCF5CF0ECCF5DF018C05EF0182ACAE3D3
:1019F00012001E0E5F5CD8A485D060521AE1226AE4
:101A00004B6A4A6A616A4D6A4C6A626A4F6A4E6AF8
:101A1000636A516A506A646A536A526A656A556AAF
:101A2000546A666A576A566A676A596A586A686A7F
:101A300068D060C061F003EE8DF0D8906034E92684
:101A4000000EEA22EECF4AF0EFCF4BF060C062F01A
:101A500003EE8DF0D8906034E926000EEA22EECF36
:101A60004CF0EFCF4DF060C063F003EE8DF0D890F6
:101A70006034E926000EEA22EECF4EF0EFCF4FF0B1
:101A800060C064F003EE8DF0D8906034E926000E5B
:101A9000EA22EECF50F0EFCF51F060C065F003EED8
:101AA0008DF0D8906034E926000EEA22EECF52F095
:101AB000EFCF53F060C066F003EE8DF0D890603445
:101AC000E926000EEA22EECF54F0EFCF55F060C0C9
:101AD00067F003EE8DF0D8906034E926000EEA221C
:101AE000EECF56F0EFCF57F060C068F003EE8DF008
:101AF000D8906034E926000EEA22EECF58F0EFCFFE
:101B000059F07AD01F0E5F5C03E160C08AF074D098
:101B1000420E5F5CD8A44FD06052D8A44AD0216A4C
:101B2000206A226A00EE69F0200EEE68E82EFDD7EA
:101B30005E6889948992899089968998899A8A9E03
:101B40008A9C8A9A8A988A968A948A928A908B9A90
:101B50008B984B6A4A6A4D6A4C6A4F6A4E6A516A60
:101B6000506A536A526A556A546A576A566A596A81
:101B7000586A616A626A636A646A656A666A676A01
:101B8000686A3B6A3A6A3D6A3C6A3F6A3E6A416AF1
:101B9000406A436A426A456A446A476A466A496AD1
:101BA000486A236A896B8A6B276A266A256A246ACF
:101BB00001D0236821D07B0E5F5C1EE1216A206A80
:101BC000226A89948992899089968998899A8A9EAD
:101BD0008A9C8A9A8A988A968A948A928A908B9A00
:101BE0008B98276A266A256A246A00EE69F0200E1F
:101BF000EE68E82EFDD75E685F681200186A800EF6
:101C0000185C1AE21850D00DF3CF0DF0F4CF0EF09F
:101C10000E260D50FF08006EFF0E0E54016E03EEEF
:101C20008DF0D8901834E926000EEA2200C0EEFFAD
:101C300001C0EFFF182AE3E31200010E02018E6FCC
:101C4000F40E8D6F010E186E0001800E185C2DE2EF
:101C5000060E0E6E7C0E0D6E106A280E0F6E126A46
:101C600018C011F01106000E125A10C00BF00FC070
:101C70000AF012C007F011C006F025EC00F00F6E5C
:101C800009C010F00F500D24006E10500E20016E90
:101C900002EE8DF0D8901834E926000EEA2200C03A
:0E1CA000EEFF01C0EFFF182ACFE31200FFD7BE
:020000040030CA
:0300010006160ED2
:020005008580F4
:060008000FC00FE00F40E5
:00000001FF
